:020000007F2857
:080008006B2882070034453427
:1000100001345434FF34203482070034493402342C
:10002000413401344E3403344D34FF3420348207DC
:1000300000345334043455340234523406345734C3
:100040000134443405344B340334473407344F34DB
:10005000FF342034820700344834083456340434E2
:10006000463402344C34063450340E344A340134AD
:10007000423409345834053443340D34593403348C
:100080005A340B345134FF34203482070034353471
:1000900010343434183433341C3432341E34313494
:1000A0001F343034013436340334373407343834B1
:1000B0000F34393411343D34FF342034820728346E
:1000C00023340C343F3421342D342A342E34333449
:1000D0002C34FF342034A200030EA300920A930AAA
:1000E000950A0A301502031C77289501940A64309A
:1000F00081000B11230E8300A20E220E0900850140
:1001000086018316FF3085000030860001148110BF
:100110000115811181128312643081008B168B17B7
:10012000A101A001A0140F309C009D0026309E006C
:10013000FF3096009700980099009A009B0092016A
:10014000930191019001940195019F0108308E0067
:100150002030AA005030AB00A621C721A723A72337
:10016000851CB328B72841226400851CB428051CCF
:10017000CF282018AF282014A0109201EB221D08D0
:100180001302031CAE28E520F220051DAE281E0830
:100190001302031CAE2820308F006923AE28A01C58
:1001A000DA28C8301302031CAF289301F22008306C
:1001B0008E00AF28A01420109301DF22A10A0F3077
:1001C00021020318AD227B22AE2808300E02031C48
:1001D000F0288E0191080319EE28CB229401950195
:1001E0008E0A08002030A40091080319080001308D
:1001F0009102031DFD2822211C2902309102031DBA
:10020000032938211C2904309102031D09294E219C
:100210001C2908309102031D0F2964211C2910306C
:100220009102031D15297A211C2920309102031DFA
:100230001B2990211C292A30A4008F0091019001D4
:10024000692308000301A5000520A600FF3026024F
:10025000031D2C292A3036292608100203193329B8
:100260002508023E23292508013E0520A400080098
:100270000301A5000C20A600FF302602031D422921
:100280002A304C2926081002031949292508023E64
:1002900039292508013E0C20A40008000301A5000F
:1002A0001720A600FF302602031D58292A30622994
:1002B0002608100203195F292508023E4F29250848
:1002C000013E1720A40008000301A5002A20A60073
:1002D000FF302602031D6E292A30782926081002D5
:1002E000031975292508023E65292508013E2A20A3
:1002F000A40008000301A5004520A600FF30260247
:10030000031D84292A308E292608100203198B29FF
:100310002508023E7B292508013E4520A40008004F
:100320000301A5005E20A600FF302602031D9A29C6
:100330002A30A429260810020319A1292508023E03
:1003400091292508013E5E20A40008003130860076
:1003500006109D233130860006109D233130860023
:1003600006109D232130860006109D232830AC0006
:100370005C239D230630AC005C239D230C30AC0035
:100380005C239D230130AC005C239D2308002030BA
:10039000A6002A30A7002030A8000330A500532370
:1003A0004330A6005730A7002030A8000330A50036
:1003B00053234430A6004530A7004330A8004F30F7
:1003C000A9000430A50053234430A6004530A700FF
:1003D0005230A8000330A50053232030A6002A3055
:1003E000A7002030A8000330A50053232030A6002A
:1003F0006230A7007930A8002030A9000430A500A1
:1004000053236930A6006B30A7003330A8006F304B
:10041000A9000430A50053236930A6006C30A70062
:100420002030A8002030A9000430A500532320303C
:10043000A6002030A7007E30A8002030A90004309C
:10044000A500532308002908A400A5016430A402D4
:1004500003182C2AA4072E2AA50A272A2508303893
:10046000A6000A30A501A4020318382AA4073A2AD4
:10047000A50A332A25083038A70024083038A800F8
:1004800008002030A6002030A7000230A50053232A
:100490001F08A900232226080F39031D512A2030E6
:1004A000A6000330A50053232030A6006330A70028
:1004B0006830A8006130A9000430A50053237230D1
:1004C000A6002F30A7006D30A8006930A9000430C5
:1004D000A50053236E30A6002030A7002030A800CE
:1004E0000330A500532320308F001030A50069236E
:1004F000A50B772A08001118832A11141C08120270
:1005000003181014AC2A91188B2A91141C0812029B
:1005100003189014AC2A1119932A11151C08120201
:1005200003181015AC2A91199B2A91151C08120268
:1005300003189015AC2A111AA32A11161C081202CE
:1005400003181016AC2A911AAB2A91161C08120235
:1005500003189016AC2A111708001808A7000230DB
:10056000A800352327089C001B08A7000230A8001C
:10057000352327089D001B08A7000530A800352358
:1005800027089E00A101FF3096009700980099006F
:100590009A009B0008000A30A7000830A800352305
:1005A0003C30A80035231408A80042232708270759
:1005B00014020318DC2AA60A26089F00080003304C
:1005C0001202031CEA2A12081802031CEA2A120863
:1005D0009800F722080003301302031CF62A1308C0
:1005E0001B02031CF62A13089B0016230800170899
:1005F00018020318012B1708A600180897002608F0
:100600009800160817020318152B1608A6001708DD
:10061000960026089700170818020318152B1708CC
:10062000A600180897002608980008001A081B0260
:100630000318202B1A08A6001B089A0026089B0006
:1006400019081A020318342B1908A6001A08990071
:1006500026089A001A081B020318342B1A08A60051
:100660001B089A0026089B000800A6012708A50081
:10067000A80364002508A707031C3F2BA60AA80BA4
:10068000392B0800A5016400A50A2808A702031851
:10069000432B0130A6020318432B2808A707A50304
:1006A0002508A60008002630840000088F00692372
:1006B000840AA50B552B08002C08F0390138860058
:1006C0000610B1232C0EF039013886000610B12334
:1006D00008002A088038AC005C230F08F039033882
:1006E00086000610B1230F0EF0390338860006107D
:1006F000B1232B088038AC005C230F08F039033895
:1007000086000610B1230F0EF0390338860006105C
:10071000B1231830AC005C232A08273C0319922B24
:10072000AA0A942B0030AA002B08673C03199A2BC5
:10073000AB0A9C2B4030AB0008007D308C0064304D
:100740008D0064008D0BA12B8C0B9F2B080030308B
:100750008C0019308D0064008D0BAB2B8C0BA92BFA
:10076000080014308C00640000008C0BB32B0800D0
:02400E00FD3F74
:00000001FF
